:020000040800F2
:10000000081A0020F93500081D0400081F04000824
:100010002104000823040008250400080000000053
:10002000000000000000000000000000270400089D
:1000300029040008000000002B0400084105000806
:100040004D3600085136000855360008593600086C
:100050005D3600086136000865360008693600081C
:100060006D3600087136000875360008570D000817
:100070007D3600088136000885360008893600087C
:100080008D3600089136000895360008993600082C
:100090009D360008A1360008A5360008A9360008DC
:1000A000AD360008B1360008B5360008B93600088C
:1000B000BD360008C1360008C5360008C93600083C
:1000C000CD360008D1360008D5360008D9360008EC
:1000D000DD360008E1360008E5360008E93600089C
:1000E000ED360008F1360008F536000840B2002869
:1000F00009D540B210F00F00DFF86C238018090119
:1001000000F8041C04E040B2DFF8602309018154C8
:10011000704780B5B0F1807F01D3012013E0000269
:10012000000A401EDFF8481308600F215FF0FF301F
:10013000FFF7DCFFDFF83C0300210160DFF8380344
:1001400007210160002002BD80B5DFF830030068A0
:1001500050F00100DFF824130860DFF82403006882
:10016000DFF820130840DFF818130860DFF80C03ED
:100170000068DFF814130840DFF800130860DFF8A8
:10018000FC02006830F48020DFF8F0120860DFF82D
:10019000F002006830F4FE00DFF8E4120860DFF8D7
:1001A000EC025FF41F01016000F006F8DFF8E002E6
:1001B0005FF00061016001BD80B500F001F801BD94
:1001C00082B00020019000200090DFF8B0020068AB
:1001D00050F48030DFF8A4120860DFF8A002006855
:1001E00010F4003000900198401C01900098002805
:1001F00003D10198B0F5A06FEFD1DFF8800200685D
:10020000800302D50120009001E0002000900098BA
:1002100001285FD1DFF87C02006850F01000DFF8A1
:1002200074120860DFF86C02006880088000DFF854
:1002300064120860DFF85C02006850F00200DFF82A
:1002400054120860DFF83802DFF8341209680160E0
:10025000DFF82C02DFF8281209680160DFF82002BD
:10026000006850F48060DFF818120860DFF81002B0
:10027000006830F47C10DFF808120860DFF8000234
:10028000006850F4E810DFF8F8110860DFF8EC01BE
:10029000006850F08070DFF8E4110860DFF8DC01DE
:1002A00000688001FAD5DFF8D80100688008800076
:1002B000DFF8CC110860DFF8C801006850F00200D8
:1002C000DFF8BC110860DFF8B801006810F00C001E
:1002D0000828F8D102B07047DFF8A001006850F09C
:1002E0000100DFF898110860DFF894010068DFF87A
:1002F00094110840DFF888110860DFF88001006879
:10030000DFF884110840DFF874110860DFF86C0131
:10031000006830F48020DFF864110860DFF86001C5
:10032000006830F4FE00DFF858110860DFF85C0167
:100330005FF41F0101607047DFF84011096831F474
:100340008031DFF838211160DFF83011096831F4AD
:100350008021DFF828211160B0F5803F03D0B0F58F
:10036000802F09D011E0DFF81401006850F48030CC
:10037000DFF80811086008E0DFF80001006850F4B9
:10038000A020DFF8F8100860FFE77047DFF8E811F9
:10039000C0B2086070470022DFF8E4301B681A0022
:1003A00032F47C1208430243DFF8D4000260704745
:1003B000DFF8C811C0B2086070470021DFF8C02024
:1003C00012681100890889000143DFF8B400016058
:1003D00070470021DFF8A8201268110031F0F00109
:1003E0000143DFF89C00016070470021DFF8902096
:1003F0001268110031F4E0610143DFF8840001600C
:1004000070470021DFF878201268110031F4605144
:1004100051EAC001DFF86800016070477047FEE7ED
:10042000FEE7FEE7FEE7704770477047816851F0CE
:1004300008018160704700218068000701D5012113
:1004400000E000210800C0B27047816851F004014B
:100450008160704700218068400701D5012100E0DC
:1004600000210800C0B2704718ED00E000E400E091
:1004700014E000E018E000E010E000E000100240AE
:10048000041002400000FFF8FFFFF6FE08100240D3
:1004900008ED00E00020024000210022C30003D547
:1004A000DFF854150A6802E0DFF8A8170A6802426C
:1004B00001D0012100E000210800C0B27047C10056
:1004C00003D5DFF83015086002E0DFF82415086076
:1004D000704710B4002100220F23C478002C21D0D3
:1004E000DFF87417096811F4E061D1F5E061090AD9
:1004F000D1F10402CB404178914082781A401143F7
:1005000009010278DFF85437D15401784911DFF836
:1005100050270123007810F01F0013FA00F042F872
:1005200021000BE001784911DFF8F827012300785A
:1005300010F01F0013FA00F042F8210010BC7047C1
:10054000DFF8E4070068401CDFF8DC17086070473C
:1005500010B504004FF4E150FFF7DBFDDFF8C807EA
:1005600000210160DFF8C0070068A042FAD3DFF87D
:10057000C0080021016010BD0000424260004242FC
:10058000BC48006850F00100BA490860B9480068EA
:1005900050F00800B7490860DFF89007006850F095
:1005A0000070DFF888170860DFF88808006850F0EE
:1005B0000050DFF880180860DFF87808006830F035
:1005C0008050DFF870180860DFF868080068800065
:1005D0008008DFF860180860DFF85808006850F0FD
:1005E0000070DFF850180860DFF84808006830F045
:1005F0008070DFF840180860DFF83808006830F0D5
:100600004060DFF830180860DFF82808006850F410
:100610000010DFF820180860DFF81808006830F4D0
:100620008010DFF810180860DFF80808006830F460
:100630004000DFF800180860DFF8F807006850F4A1
:100640000030DFF8F0170860DFF8E807006830F4E2
:100650008030DFF8E0170860DFF8D807006830F472
:100660004020DFF8D0170860DFF8C807006850F4B2
:100670000050DFF8C0170860DFF8B807006830F4F2
:100680008050DFF8B0170860DFF8A807006830F482
:100690004040DFF8A01708607047000080B5DFF821
:1006A0009807006850F48010DFF88C170860DFF8B6
:1006B0008807006850F40020DFF87C1708600A20E3
:1006C000FFF746FFDFF87007006850F00800DFF81A
:1006D000681708600A20FFF73BFF0121E22000F0C5
:1006E00025F80A20FFF734FF0121AF2000F01EF8A3
:1006F0000121A42000F01AF801212F2000F016F8A3
:100700000121B02000F012F80121102000F00EF8B5
:100710000121002000F00AF80121902000F006F8E5
:100720000121A12000F002F801BD0000DFF8082738
:10073000126852F48002DFF800371A60DFF8F826FA
:10074000126852F48012DFF8F0361A60C9B201293B
:1007500008D1DFF8E416096851F40011DFF8D82653
:10076000116007E0DFF8D016096851F02001DFF8CA
:10077000C8261160DFF8C016096851F04001DFF8A3
:10078000B8261160DFF8B016096851F48001DFF86F
:10079000A8261160002119E0DFF89C26126852F4A7
:1007A0000012DFF894361A60DFF88C26126852F0D7
:1007B0004002DFF884361A60DFF87C26126852F4B3
:1007C0008002DFF874361A604000491CC9B208295B
:1007D0000DD210F08002D2B2802ADDD1DFF8582687
:1007E000126852F02002DFF850361A60DCE7DFF8BA
:1007F0004806006850F40010DFF83C1608607047A7
:1008000038B50121B020FFF791FF01211020FFF73B
:100810008DFF01210020FFF789FF00240CE0022159
:10082000602000FB0450DFF81426805CFFF77EFF99
:100830006D1E002DF3D5641C092C01DA5F25F8E745
:1008400031BD80B5002004E0DFF8F01500224254ED
:10085000401CB0F5587FF7DBFFF7D2FF01BD002049
:1008600004E0DFF8D81500224254401CB0F5587F50
:10087000F7DB70471810024010B4C0B261282FD2C5
:10088000C9B249292CD2C9B2082391FBF3F36024E1
:10089000C0B204FB0300C9B20B00DBB2082493FB17
:1008A000F4F3B1EBC301DFF89435C35CD2B2002A94
:1008B00004D1012212FA01F18B430EE0D2B2012AD7
:1008C00004D1012212FA01F10B4306E0D2B2022A4E
:1008D00003D1012212FA01F14B40DFF860154354B5
:1008E00010BC7047C9B2491E6022C0B2401E062328
:1008F000584302FB0100DFF87019086070470020C0
:1009000005E0C0B2DFF8641900224254401CC0B2B6
:100910001328F6D3704710B480281CDB0021C9B21D
:10092000052934D20522C9B202FB0012DFF81035C6
:10093000D218B2F570721278DFF82C391B68DFF824
:10094000FC441A55DFF820291268521CDFF81839C8
:100950001A60491CE3E7002116E00522C9B202FB38
:100960000012DFF8E034D21812F8A02CDFF8F838C3
:100970001B68DFF8C8441A55DFF8EC281268521CCF
:10098000DFF8E4381A60491CC9B20529E5D3DFF85D
:10099000D8080068DFF8A41400224254DFF8C80821
:1009A0000068401CDFF8C018086010BC704710B524
:1009B000C0B2122802D2C9B2092900D317E0C9B2C5
:1009C000C0B2FFF78FFF00240CE0E4B2DFF89C0810
:1009D000205C002805D0E4B2DFF89008205CFFF727
:1009E0009AFF641CE4B2112CEFD3FFF788FF10BD0F
:1009F00004000240040402400004024080B5CC48D8
:100A0000006850F00400CA490860DFF86408006814
:100A100030F44050DFF858180860DFF854080068D8
:100A200030F44040DFF848180860C148006850F4CE
:100A30000070BF490860DFF83C08006850F440408F
:100A4000DFF830180860DFF83008006850F0010067
:100A5000DFF824180860DFF82008006850F4000070
:100A6000DFF814180860DFF81008006830F4602020
:100A7000DFF804180860DFF80008006830F4801020
:100A8000DFF8F4170860DFF8F407006850F46060DE
:100A9000DFF8E8170860DFF8E007006850F48070BE
:100AA000DFF8D4170860DFF8D807006850F470004A
:100AB000DFF8CC170860DFF8C40747F6F87101606B
:100AC000DFF8C0075FF47C010160DFF8B807006859
:100AD00050F46000DFF8AC170860DFF8A00700688A
:100AE00050F46060DFF894170860DFF89C07006836
:100AF00050F01100DFF890170860DFF88C070068ED
:100B000050F06000DFF880170860DFF87C070068AD
:100B100050F44060DFF870170860DFF86C07006879
:100B200050F4C030DFF860170860DFF85C07006839
:100B300050F44010DFF850170860DFF84C070068E9
:100B400050F0C060DFF840170860DFF84007006829
:100B500050F00300DFF834170860DFF83007006852
:100B600050F06000DFF824170860DFF82007006805
:100B700050F44060DFF814170860DFF810070068D1
:100B800050F4C030DFF804170860DFF80007006891
:100B900050F44010DFF8F4160860DFF8F006006843
:100BA00050F0C060DFF8E4160860DFF8D406006893
:100BB00050F00300DFF8C8160860DFF8C4060068CC
:100BC00050F06000DFF8B8160860DFF8B40600687F
:100BD00050F44060DFF8A8160860DFF8A40600684B
:100BE00050F4C030DFF898160860DFF8A4060068FB
:100BF00050F48070DFF898160860DFF87C06006813
:100C000050F40000DFF870160860DFF86C0600682A
:100C100050F00200DFF860160860DFF87806FFF792
:100C200005FCDFF87006FFF706FC0028F9D1DFF8B5
:100C30006406FFF70AFCDFF85C06FFF70BFC0028F0
:100C4000F9D1DFF83406006850F48000DFF8281688
:100C5000086001BD000002400CED00E000E400E08F
:100C600000E100E0DFF83006006850F00100DFF836
:100C700028160860DFF82406DFF824160160DFF884
:100C80002406DFF824160160DFF82006006830F043
:100C90001000DFF818160860DFF814064021016024
:100CA000DFF80806006830F04000DFF80016086042
:100CB000DFF8F805006850F08000DFF8F0150860F4
:100CC000DFF8E805006850F48070DFF8E015086090
:100CD000DFF8D805006850F48060DFF8D0150860B0
:100CE000DFF8C805006850F44050DFF8C015086010
:100CF000DFF8B805006850F00200DFF8B0150860B2
:100D0000DFF8A805006850F02000DFF8A0150860A3
:100D1000DFF89805006850F00100DFF890150860D2
:100D20007047000080E100E0F80D00200400014061
:100D30001810024080B50B208DF8000000208DF8BF
:100D4000010000208DF8020001208DF8030000A8AA
:100D5000FFF7BFFB01BD38B500240220FFF79CFB65
:100D6000002860D0DFF84C050068401CDFF844150F
:100D70000860DFF844050021016000200BE0DFF887
:100D800038150968DFF8202532F810205118DFF8EF
:100D900028251160401C402821DA002801D00121BB
:100DA00000E00021102801D0012200E000222028CC
:100DB00001D0012300E00023302801D0012500E00C
:100DC0000025C9B2D2B21140DBB21940EDB22942BE
:100DD000D5D0DFF8D41431F810100C19DAE7DFF8A9
:100DE000D80400688008DFF8D0140860002000FBF9
:100DF00004F06421B0FBF1F004193C20B4FBF0F4E2
:100E0000DFF8B80404604FF4C0700AE0DFF8AC14F7
:100E100011EB800151F8041CDFF8A02442F82010E7
:100E2000401E0128F2DA0120FFF749FB31BD000026
:100E300010E000E0000C0140100C0140700900209F
:100E4000E001002000000020E2B0DFF874940020F0
:100E50000090FFF741FA0020FFF76EFA0120FFF73C
:100E600095FA0020FFF7B5FA0020FFF7BEFA002040
:100E7000FFF7C7FA00210020FFF78DFA0020FFF7E7
:100E80009CFA0120FFF794FADFF83804006850F06C
:100E90000100DFF830140860FFF74CFFFFF770FB2C
:100EA000FFF7FCFBFFF7CDFCDFF81C04802101609D
:100EB000DFF81814DFF8B40300F02EFA0521012042
:100EC000FFF775FDFFF71BFDFFF79AFC4FF4C870A5
:100ED000FFF73EFBFFF792FDFFF7C4FEDFF8D403F8
:100EE00000210160DFF8CC0300686028FADBDFF83E
:100EF000E0030090DFF8C003006800F027FA01006B
:100F0000009800F049FA0090DFF8B003406800F064
:100F10001DFA009900F0BEFA81460098494600F09B
:100F200025FBDFF8B0130860DFF8A8030068DFF8DE
:100F3000A81300F05DFB0DD8DFF8A013CB4800F03C
:100F4000EBF905210120FFF732FDFFF7D8FCFFF791
:100F500057FCFEE75FF0000805E001A8002140F81B
:100F6000281018F10108B8F5C07FF6D3DFF8700338
:100F7000002101600EE001220F214046C0B2FFF7C0
:100F80007BFC18F10108B8F1600FF4D3FFF738FCCF
:100F9000FFF765FC1F2C3ED33000390000F03AFB10
:100FA0005FF0804100F0F8F9390000F0DFFACD4938
:100FB00008603000390000F02DFBCB4900F018FB31
:100FC00000D80024C7480068C84900F0E5F9C749BF
:100FD00000F060FAC2490860C1480068C44900F0E6
:100FE0009DFB03D2BE480021016006E0BC480068BA
:100FF000C04900F0BBFABA4908603000390000F07F
:1010000009FBB94900F0F4FA05D8BB48310000F0FB
:10101000ADFAB34908605FF0000888E0AC48009082
:10102000A548006800F092F90100009800F0B4F9BA
:101030000090A24850F8280000F088F9009900F0CC
:1010400029FA81464846A349096800F0E3FA814637
:10105000AA48494600F01EFA8146484600F070FB57
:1010600001A941F82800B8F1000F08D14D460198B8
:1010700000F06CF90600019800F068F9070001A87B
:1010800050F8280000F062F90100300000F046FB43
:1010900005D201A850F8280000F058F9060001A870
:1010A00050F8280000F052F9390000F037FB05D263
:1010B00001A850F8280000F049F9070088480068A6
:1010C0008F4900F053FA310000F028FB00D2641C75
:1010D00038008349096800F021FB00D2641C4846AF
:1010E0007F49096800F096FA864900F055F9814673
:1010F0004846002100F07CFA17D201200421B8FBF9
:10110000F1F202FB1182002A0FD1C0070DD5012296
:101110009246484600F026FBD0F140015246C9B243
:101120005FEA9800C0B2FFF7A7FB18F10108B8F515
:10113000C07FFFF473AF6A480068714900F016FA87
:10114000310000F0EBFA00D2641C380064490968F1
:1011500000F0E4FA00D2641C5FF0000809E001220C
:1011600040214046C0B28000C0B2FFF785FB18F1B5
:101170000108B8F1180FF2D35FF0000809E001226E
:1011800030214046C0B24000C0B2FFF775FB18F1F5
:101190000108B8F1300FF2D35FF0000809E0012236
:1011A00020214046C0B28000C0B2FFF765FB18F1B5
:1011B0000108B8F1180FF2D34948006800F0C0FAEE
:1011C00010F164025049294800F0A6F804210C20CF
:1011D000FFF7EDFBFFF793FB4148006800F0B0FA22
:1011E00002004949214800F097F808210C20FFF738
:1011F000DEFBFFF784FB3000390000F00BFA80467D
:1012000042491A4800F088F801210120FFF7CFFB7E
:10121000FFF775FB380000F093FA0090300000F003
:101220008FFA03009946280000F08AFA02004B4624
:1012300037490E4800F070F802210120FFF7B7FB94
:10124000FFF75DFB404600F07BFA0200314907489A
:1012500000F062F803210120FFF7A9FBFFF74FFB25
:101260005FF000088FE60000FC0D0020C80D002094
:1012700000080140041002400824014010240140ED
:101280002C2401400C24014034240140302401402E
:1012900004240140002401401410024010000240C8
:1012A0004C24014014000240D00C002008000240F1
:1012B0000C000240E40D0020E80D00207003002027
:1012C00000008C4218100240140C0140C835000880
:1012D0009A99993FF40D0020CDCCCC3CD83500082C
:1012E000F00D0020EC0D00200100C842000020415C
:1012F00000004842000048C20000C8C200A0E74405
:101300000000C8420000404020360008B435000804
:10131000E8350008083600080CB41CB5044604A8DB
:101320000190009401AB0A4600A9074878441830A0
:1013300000F03AFA009900220A7000285CBF009879
:10134000001B16BC5DF80CFBDB140000002800BF7E
:101350000AD0B0FA80F18840D1F19D01C90502069A
:1013600072F1004241EB1020704710B450F8041B9A
:1013700081B102681218001D50F8043BDC0744BF1D
:10138000A9F10104E31852F8044B43F8044B091F78
:10139000F9D1EBE710BC704710B5FF2313EAD05426
:1013A0001DBF13EAD1529C429A4239E0A41ADA07CF
:1013B00080EA0103134042EA012142EA0020421A76
:1013C0003CBF641E01EB4202090AB2FBF1FE01FBC5
:1013D0001E221202B2FBF1F001FB10226EF30F206D
:1013E0001202B2FBF1FE4EEA00207F3406DDFE2C35
:1013F00024DA53EA500050EBC45010BDD4F102047B
:1014000001FB1E2240F08071192C1DDC21FA04F032
:10141000C4F12004A140114371F10042584110BDB4
:101420009C421ABF03EAD1529A420FE080EA010EB1
:101430000EF00043400004D0490016D143F0FF40B5
:1014400010BD490008BFD343180010BD9C4205D110
:10145000D21AF7D001F00041484010BD4A0212BF35
:101460000846484000F0004010BD4AB90902B1FAF0
:1014700081F2914044B1A418C00140F000409EE7C1
:10148000C90141F0004152420002B0FA80F4A0408C
:10149000141B94E7FF2212EAD05C1DBF12EAD1535D
:1014A000944593422BE09C44D30780EA01021A4002
:1014B00043EA002043EA0121A1FB0030410038BF8C
:1014C00040007CF17F010BDBFE294ADA5B0842EA2F
:1014D000C15153EA006373F1004C51EB1020704787
:1014E000D1F1080CDCF120012FDB5B0810FA01F1CF
:1014F0000B4373F1004120FA0CF0504170479445C2
:101500001CBF02EAD153934280EA010202F000427A
:101510001DD0400019D0490017D05BB9634514D0E5
:101520000902B1FA81F39940BCEB030CC00140F011
:101530000040C1E70002B0FA80FC10FA0CF0B3EBF7
:101540000C0CC90141F00041B6E7100070474000A3
:101550000AD0490008D010F1807F94BF11F1807F3C
:1015600002E042F0FF407047D043704790EA010F1D
:1015700044BF81F0004100F055B800BF421A3CBFA3
:10158000801A89184FF0004CC0F3C752FF2A24D0AC
:10159000C1F3C75313B3D21AD2F1190327DD4CEAB2
:1015A00001214CFA03F321EA0303D140C20D4CEAB6
:1015B0000020401834BF20EA0C004CEA5000D2054D
:1015C00053EA006373EB0C0C52EB1020420012F153
:1015D000807F38BF7047C00DC0057047490212BFF9
:1015E0009A4200EB5120F8E7D2F11703D9D57047A2
:1015F0004FF0807C1CEB400F94BF1CEB410F05E0CB
:1016000040EA010C5FEA4C0C01D28142704718BFDE
:101610008842704790EA010F44BF81F00041FFF714
:10162000ADBF00BF431A4FF000423EBF5340C01A47
:10163000C91800BFD3095FEAD05C13EB400F34BF79
:10164000B3EB410F40E07CEBD1530CD342EA0121D4
:1016500022D8D1EB402009D3400A28BF5FEA5001CD
:1016600040EBCC507047401A15D04002B0FA80F2DF
:10167000521C9040400A4FEA3C23B3EB026384BF04
:1016800000EB730007E040F400001A16DB07C2F11C
:101690000102D04018437047182BFCDC31FA03F2EA
:1016A00002FA03F3591A38BF42F00102D2EB40208C
:1016B0003CBF4000ACF1010C5FEACC5CC20572F1AA
:1016C00000414CEB5020704713EB400F0FD24B0002
:1016D00009D0ACEBD153022B03DB4902172BDDDD24
:1016E00070479143401A4300D5D10020704713EB57
:1016F000410FD0D36FF00000704750F8041B61B168
:1017000050F8042BD30744BFA9F101039A18002312
:1017100042F8043B091FFAD1EFE770474FF0807C95
:101720001CEB400F94BF1CEB410F05E040EA010C9D
:101730005FEA4C0C01D28842704718BF8142704763
:1017400040000DD2010E7F390AD4D1F11F0104D41B
:10175000C00140F00040C84070477FF00000704773
:10176000002070474100090E7F3915D4D1F11F01C7
:1017700014D4400007D2C00140F00040C84048BF28
:101780006FF000407047C00140F00040C8404CBFBF
:101790004FF00040404270470020704700424FF039
:1017A000004058BFC04370472DE9F04FA5B08046B8
:1017B00015461E460FF2B050D0E90023CDE91223A2
:1017C000049104AF0020786214AC6FF0004900E08F
:1017D00055440020ADF8020012AB4FF0FF3229460D
:1017E0000DF1020001F00DF88246BAF1010F08DA9E
:1017F0002878B0F1010A6AEB0A0A6FEA0A004FEA98
:10180000D07ABDF8020025280CBFAAF10103534687
:10181000012B07DB2A4602A9404600F0CEFF002834
:1018200000F1E780BDF80200252807D10020F8600C
:1018300038617861B861F861386205E00028C7D185
:10184000786A99E240F0010015F8011F2029F9D0CB
:1018500023290DD02B2904D02D2906D030290AD0D8
:101860000CE040F0020080B2EEE740F00400FAE73E
:1018700040F00800F7E740F01000F4E72A290DD106
:1018800031680A1D32600968F962002904D54942AD
:10189000F96240F0040080B26D1C12E00021F96290
:1018A00009E0F96A494505D001EB810302EB4301E8
:1018B0003039F9626D1C2A78A2F13001C9B20A29C7
:1018C000EFD329782E2903D04FF0FF31B9621DE004
:1018D00015F8011F2A2906D131680A1D32600968EE
:1018E000B9626D1C12E00021B96209E0B96A49458C
:1018F00005D001EB810302EB43013039B9626D1C65
:101900002A78A2F13001C9B20A29EFD338862978A2
:101910000FF25C4000F08AFF08B115F8010B8DF85A
:1019200042009DF84200682804D1287868280AD12E
:10193000622005E06C2804BF28786C2803D1712050
:101940008DF842006D1C14A8B8602978B1F125000B
:1019500027D01C3800F08680001F022840F28280C9
:10196000133800F0A98009387CD0801E00F03A813D
:10197000401E00F0E480401E022873D9001F00F0D2
:10198000DE80401F43D0401E00F09680401E33D0C2
:10199000C01E0BD0801E00F08F80C01E00F08C8017
:1019A00040E1F868411CF960252144E19DF84200BE
:1019B0006C28306813D0011D316000687860BA6A05
:1019C000002A02D500F03EFF07E0002100F056FF9C
:1019D00000281ABF7968401AB86A38612CE1011DE5
:1019E0003160026802A9404600F0C9F9002840F1C0
:1019F00023814FF0FF30BFE13068011D3160006886
:101A00000021CDE9020114A878607821E6E09DF874
:101A10004200622818D0682806D06A280BD06C28AB
:101A200019D0712807D016E03068011D3160796A3D
:101A30000068018000E13268101D3060786AC117CB
:101A40001268C2E90001F7E03068011D3160796A6F
:101A500000680170F0E03068011D3160796A00684B
:101A60000160E9E03068C01D20F00700306000F13F
:101A700008023260D0E90023CDE90223002B04D50F
:101A8000F868421CFA602D220DE0388E820704D5DA
:101A9000F868421CFA602B2205E0C00704D5F868FC
:101AA000421CFA6020220255F86814AA8018786057
:101AB00002A800F05BFBBFE09DF842006C2808BF65
:101AC000326811D0712808BF326802D06A283268A3
:101AD0000AD1D21D22F00702326094460CF10802AE
:101AE0003260DCE9002303E0131D33601268002339
:101AF000CDE90223682808BF92B207D0622808BF48
:101B0000D2B203D0742818BF7A2802D10023CDE9BD
:101B1000022397F8300000075CD5DDE90223002B93
:101B200008BF002A56D041F02000782852D1F8682A
:101B300030220255401C421CFA6001554AE09DF8D3
:101B4000420062280CD0682810D06A281AD06C286D
:101B500023D0712816D074281FD07A280CD01CE00E
:101B60003068021D326090F900201AE03068021DD2
:101B70003260B0F9002014E03068021D3260026863
:101B800000230FE03068C01D20F00700306000F136
:101B900008023260D0E9002304E03068021D3260A0
:101BA0000268D317CDE90223002B04DAF868421C3F
:101BB000FA602D220DE0388E820704D5F868421CA9
:101BC000FA602B2205E0C00704D5F868421CFA60D1
:101BD00020220255F86814AA8018786002A800F044
:101BE0003AFA29E09DF842006C2807D0F868411CB9
:101BF000F96031680A1D326009681CE03068011D17
:101C000031600068ADF804000020ADF806004FF028
:101C1000FF30B86201AA02A9404600F0B0F80028DF
:101C20000AD5E6E6F868421CFA602522025519B189
:101C3000F868421CFA6001556D1CF86AF968401A90
:101C4000B969401A3969401AF969401A7969401A24
:101C5000396AA0EB010A97F83000400712D420201F
:101C60008DF80000BAF1010F0CDBD346012300AA66
:101C700002A9404600F0A1FD00287FF4BAAEBBF1F6
:101C8000010BF3D1FB6814AA02A9404600F095FDB0
:101C900000287FF4AEAE30208DF80000D7F818B0E1
:101CA000BBF1010F0BDB012300AA02A9404600F0A3
:101CB00084FD00287FF49DAEBBF1010BF3D13B699D
:101CC0007A6802A9404600F078FD00287FF491AEC2
:101CD00030208DF80000D7F81CB0BBF1010F0BDBF2
:101CE000012300AA02A9404600F067FD00287FF406
:101CF00080AEBBF1010BF3D17B693869796842187A
:101D000002A9404600F059FD00287FF472AE302051
:101D10008DF80000D7F820B0BBF1010F0BDB0123D9
:101D200000AA02A9404600F048FD00287FF461AEF9
:101D3000BBF1010BF3D197F8300040077FF549ADB7
:101D400020208DF80000BAF1010FFFF642AD01230B
:101D500000AA02A9404600F030FD00287FF449AEF9
:101D6000BAF1010AF3D134E50000000000000000E0
:101D7000686A6C747A4C000025B0BDE8F08F2DE9DC
:101D8000F04F95B083460F461446D7F830A0BAF10D
:101D9000000F48BF6FF0004A00F09CFD796B4018BF
:101DA00001900FF64422D2E90001CDE9020197F833
:101DB0003800400702D40198412805D20DF11009DE
:101DC00040200190002509E000F08AFD5FEA00094B
:101DD000F8D14FF0FF303BE1AAEB080ABAF1010F4E
:101DE000C0F2A98002AA21880DF1010000F0D0FD07
:101DF0005FEA000800F1BF80208818B9B8F1010837
:101E000000F1B980C245C0F296807869019908EB6B
:101E10000002914280F080807D634042396A401A1E
:101E2000B969401A796A401AF969401AB96A451ABB
:101E300097F83800400710D420208DF80000012DBD
:101E40000BDB2E46012300AA3946584600F0B5FCAC
:101E5000002840F09080761EF4D17B694A463946CE
:101E6000584600F0AAFC002840F0858030208DF80C
:101E700000003E6A012E09DB012300AA39465846BC
:101E800000F09BFC002876D1761EF5D1BB69FA687C
:101E90003946584600F091FC00286CD130208DF86E
:101EA00000007E6A012E09DB012300AA394658464C
:101EB00000F083FC00285ED1761EF5D1FB69B8697D
:101EC000F96842183946584600F077FC002852D18C
:101ED00030208DF80000BE6A012E09DB012300AA24
:101EE0003946584600F069FC002844D1761EF5D1E9
:101EF00097F8380040070DD520208DF80000012DFF
:101F000008DB012300AA3946584600F056FC90BB76
:101F10006D1EF6D100257D6142460DF10101786903
:101F2000484400F043FD78694044786134F8020B7E
:101F300000287FF451AF786B7969401A396A401AEA
:101F4000B969401A796A401AF969401AB96AA0EB6E
:101F5000010897F83800400712D420208DF80000BF
:101F6000B8F1010F0CDB4446012300AA394658465C
:101F700000F023FC10B14FF0FF3562E0641EF3D196
:101F80007B694A463946584600F017FC0028F2D1D2
:101F900030208DF800003C6A012C09DB012300AAE7
:101FA0003946584600F009FC0028E4D1641EF5D1FA
:101FB000BB69FA683946584600F0FFFB0028DAD1C1
:101FC00030208DF800007C6A012C09DB012300AA77
:101FD0003946584600F0F1FB0028CCD1641EF5D1FB
:101FE000FB69B869F96842183946584600F0E5FBC4
:101FF0000028C0D130208DF80000BC6A012C09DB1C
:10200000012300AA3946584600F0D7FB0028B2D178
:10201000641EF5D197F83800400710D520208DF8C0
:102020000000B8F1010F0ADB012300AA3946584627
:1020300000F0C3FB00289ED1B8F10108F4D17D6106
:102040007D6304A881451CBF484600F0EBFC284690
:1020500015B0BDE8F08F2DE9FA4782B00646356924
:102060006F2908BF082705D041F02000782814BF49
:102070000A2710273C24D6E90001804689469DF8AE
:102080000820642A18BF692A05D1002903DAD8F18B
:10209000000869EB4909B9F1000F08BFB8F1000F5A
:1020A0000CD1306B50B9082F3BD196F8380000079F
:1020B00037D53B24302085F83B0032E0A4F1010AFB
:1020C0005446FB17404649463A4600F0EBFCCDE942
:1020D0000089B846A8FB0023DDE90089A8EB0202CD
:1020E0003032D2B23A2A03D39DF80830513B9A18C5
:1020F0000AF8052080465FEA010908BFB8F1000F21
:1021000003D0F06861198842D8D3082F09D196F816
:102110003800000705D5605D302802D0641E3020ED
:102120006055C4F13C00B0616119F160316B8842C7
:1021300007DA081A3062308F4FF6EF7108403087A7
:1021400010E000290ED596F8381001F0140110297E
:1021500008D1716B7269891A326A891A081A0128C2
:10216000A8BF306204B0BDE8F08700002DE9F24F4F
:102170008EB0044604AED4E90001CDE902019DF819
:10218000380040F020008DF8000061280BD0206B53
:10219000002848BF062005D404BF9DF8000067282A
:1021A00001D1012020636168C1F30A5040F2FF733E
:1021B00098421ED1080304BF206800280AD10320DA
:1021C000A0619DF838006138C0B21A2838D30FF2E8
:1021D0002C6109E00320A0619DF838006138C0B28D
:1021E0001A282AD30FF20C610322E06800F0DEFB0C
:1021F000B9E1012817DA204600F0CBFC012812DBF8
:10220000002700209DF80010612920D1E1683022CC
:1022100001F8012B4A1CE2609DF83820612A0CBFAE
:10222000782258220FE040F2FE31626861F31E52BC
:102230006260471A4FF0FF30E4E70FF2B451D3E782
:102240000FF2B451D0E70A706169891C616110B95D
:10225000002500277EE19DF80000612840F097806E
:10226000206B00284CBF2125451C2DB26E1CD4E9E3
:102270000089DDE902010022002300F0ABFC3ABF37
:1022800089F00040CDE90280CDE902893F1F8DF839
:1022900010200DF11108012E35DBDDE902010022CD
:1022A000002300F0AFFC2ED21C2102A800F0C2FCDB
:1022B000DDE9020100F044FD8146F61F012E09DB35
:1022C00000F06AFD02460B46DDE9020100F07CFDEC
:1022D000CDE9020108F20700072105E009F00F022D
:1022E00000F8012D4FEA2919B9F1010F01DB491E50
:1022F000F4D5491E5CBF002200F8012DF9D500F28B
:102300000708012EC9DA0DF11100A8EB00010DF14B
:102310001106A942B8BF0D462DB2002D30D4284673
:10232000884206DA04A941184978082928BF0F21F4
:1023300000D2002104AA821800E06D1E401E12F88F
:1023400001398B42F9D00F2904D104A941184A78E8
:10235000521C4A70002802D504AE6D1C3F1D2DB2E0
:10236000681E0DD481190A783032D2B23A2A03D3CA
:102370009DF838303A3B9A1801F80129401EF2D5F1
:10238000206B002840F1E680681E2063E2E0DDE972
:1023900002010022002300F01DFC3CBF81F000413F
:1023A000CDE902013FB247F297507843474990FB8D
:1023B000F1F73FB2C7F107069246DFF814B1012EDC
:1023C00019DBDDE90289F00707D552465B46404636
:1023D000494600F0B9FD8046894676105046594678
:1023E00052465B4600F0B0FD82468B46002EEAD195
:1023F000CDE9028921E076429046DFF8D89012E0DC
:10240000F00707D552465B464046494600F09CFD22
:102410008046894676105046594652465B4600F043
:1024200093FD82468B46002EEAD1DDE90201424649
:102430004B4600F05BFECDE902019DF800006628E6
:102440000CBF07F10A000620216B4518142DA8BF08
:10245000132530208DF810000DF11106DFF878906B
:10246000012D3BDBDDE9020100F080FC06F10801F3
:1024700004220A26B0FBF6F303EB830EA0EB4E001A
:10248000303001F8010DB3FBF6F000EB8006A3EB52
:102490004603303301F8013D521EEAD101F108062E
:1024A000083D012DDCDBDDE9020100F05FFC00F0FE
:1024B0007DFC02460B46DDE9020100F085FC0022AE
:1024C0004B4600F041FDCDE90201CBE7A0860100BB
:1024D000000024400000F03F84D797410DF1110027
:1024E000301A0DF1110602E0401E7F1E761C317875
:1024F0003029F9D09DF80010662902D13FB2791C2D
:1025000003E065290CBF01210021226B8D182DB23B
:10251000A842B8BF05462DB2002D1BD429468142E2
:1025200004DA885D352828BF392000D230208A1986
:10253000521E00E06D1E491E12F801398342F9D087
:10254000392802D1885D401C8855002902D5761EA5
:102550006D1C7F1C3FB200972BB232469DF838109D
:10256000204600F003F80FB0BDE8F08F2DE9F047EA
:1025700086B006468A4690461C4600F0F8FE406A41
:1025800090F80090376B012C02DA01240FF27028CA
:102590004AF02000BDF93850662808BF6D1C13D0E2
:1025A000672876D16FF00300854278DBBD4276DA8A
:1025B0006D1C96F83800000702D4BC42B8BF27460D
:1025C0002DB27F1B48BF0027F068B1692DB2012DE5
:1025D00021DA4A1C30230B54012F03DA96F8381005
:1025E000090702D502F80090521CB261EF42B8BF51
:1025F0007D422DB269427162EF19A742B8BF3C46D5
:1026000024B2F46122464146B369181800F0CEF9AD
:10261000381BB062BAE00818AC4216DA22464146CE
:1026200000F0C4F9B1696118B161281B7062012F13
:1026300003DA96F83800000705D5F06801F8009035
:10264000F069401CF061B762A0E02A46414600F004
:10265000ADF9B0692818641B012F03DA96F8381019
:10266000090703D5F16800F80190401CB06124B25D
:10267000A742B8BF3C4624B2224605EB0801F368E6
:10268000C01800F093F9B0692018B061381B70626F
:102690007CE0BAF1610F14D14FF0700A16E0BC4231
:1026A00004DA96F83810090758BF27467F1E48BF3E
:1026B0000027BAF1670F14BF4FF0450A4FF0650AC3
:1026C00004E0BAF1410F08BF4FF0500AB1694A1C4B
:1026D000F06818F8013B0B54012F05DA96F8381012
:1026E000090758BFB26115D502F80090531CB361B9
:1026F000012F0FDB641E24B2A742B8BF3C4624B2B0
:1027000022464146181800F051F9B0692018B0610E
:10271000381B7062B069F16800EB010808F801AB82
:10272000002D03D42B2008F8010B03E02D2008F81E
:10273000010B6D42002402AF09E00A22294600A8DD
:1027400000F02EFE019807F8010B009D641C2DB2CD
:10275000012DF2DA022C06DA4AF02000652804BFC7
:10276000302008F8010B4CB9302008F8010B07E0C5
:10277000641E02A8205C303008F8010B012CF7DA47
:10278000B069F1684018A8EB0000F06196F83800D5
:1027900000F0140010280DD17069B1690818716A31
:1027A0000818F1690818B16A0818716B8842BCBF33
:1027B000081A306206B0BDE8F087F8B504460D4649
:1027C00016461F46002077B116F8011BA868A047DF
:1027D000A86030B1E86A401CE86200207F1EF3D197
:1027E000F2BD4FF0FF30F2BD00000000000000001D
:1027F0006E616E004E414E00696E6600494E4600A5
:102800003000F8B504460D4616461F4600F0D0FDD0
:102810003B4632462946204601B0BDE8F04000F074
:10282000DEBD0268531C0360117070470278C9B2A4
:102830008A421AB11CBF10F8012FF9E718BF002017
:102840007047000000F10103810704D010F8011B5C
:1028500089B18107FAD10268B2F10131914311F0D7
:10286000803F04BF50F8042FF6E710F8011B11B1A8
:1028700010F8011BFBE7C01A70470000C9B28307BC
:1028800006D0521E22D310F8013B9942F7D11FE027
:10289000083A13D302F1040241EA012141EA01415D
:1028A00050F8043B121F21BF4B40A3F1013C2CEA1E
:1028B000030C1CF0803FF3D0C9B2001F083210F89F
:1028C000013B521E28BF91EA030FF8D818BF012020
:1028D000401E704780B500F06BFD012002BD000076
:1028E00070B5054605F10F00C408E400C046C046B7
:1028F000A54232D2082C04D2082402E0083000F0AD
:1029000091F82248026811000CD1011D0A6802B337
:102910001368A34238BF111DF8D310E01D68A5420B
:102920000DD2191D0B68002BF8D11268011D00E0B3
:10293000191D0B6893420CD01D68A542F8D361B1F4
:102940000D682A68A2F10803A3420AD26A680A60E5
:102950000FE000F067FD0028D0D1C046C04600203F
:1029600070BD63190B606E685E60121B0B681A60A5
:102970002C60096800291DBF4A68002A091D002132
:102980000160C046C04605F1080070BDDC0D0020A6
:1029900070B504460D46164600F00AFD324629463B
:1029A0002046BDE8704000F00DBD000062B38B070B
:1029B00008D0521E11F8013B00F8013B00F02480C2
:1029C0008B07F6D1830740F0208000BF103A07D371
:1029D00030B4B1E83810103AA0E83810F9D230BC61
:1029E000530724BFB1E80810A0E8081044BF51F80D
:1029F000043B40F8043BD20724BF31F8022B20F8F7
:102A0000022B44BF0B7803707047083A07D3B1E834
:102A10000810083A40F8043B40F804CBF7D25307BB
:102A2000E4E7000000B9704710B5A0F10804206881
:102A3000082833D310F0070F30D1C046C0461848DD
:102A4000416809B18C4203D26160446017E01946C5
:102A50004B680BB1A342FAD30A6853189C421BD3AC
:102A6000A34204D123689A180A600C4607E04A681A
:102A70001AB123681B199A420ED362604C606168D8
:102A800051B1226813198B4206D1002303600868F4
:102A90008018206048686060C046C04610BD0000D5
:102AA000DC0D00201B4213D1094236D12AB18446E5
:102AB000B0FBF2F002FB10C2704700F0C7BCFCD3C1
:102AC0000022002370470B00020000210020704705
:102AD000904271EB030CF6D370B5B1FA81F4B3FAFE
:102AE00083F52C1BA340C4F1200532FA05F63343CD
:102AF000A2405FF00046E64002E05B085FEA320277
:102B0000841A71EB030524BF204629467641F4D38D
:102B100002000B003000002170BD012ACFD970B532
:102B2000140C20D0B1FA81F4B2FA82F5C4F1200479
:102B30006419B4F12006D6D3B2405FF00044F440EB
:102B4000002502E052085FEA3303C61A71EB020E59
:102B500024BF3046714664416D41F3D302000B003F
:102B60002000290070BD0C46B1FBF2F102FB1145BB
:102B70002D0445EA1045B5FBF2F402FB145580B272
:102B800040EA0545B5FBF2F002FB105240EA044072
:102B900070BD30B4436803F0004201211B031B0BDE
:102BA000436004BF0368002B08D10DE00368DD0F0C
:102BB00045EA440444605B000360491E4468E30244
:102BC000F4D523031B0B436043681A434260084655
:102BD00030BC70474FF4001C1CEB410F94BF1CEB42
:102BE000430F09E041EA030C50EA4C0C52EA0C0C8A
:102BF00003D2994208BF9042704714BF8B42824271
:102C0000704700004FF4001C1CEB410F94BF1CEBFD
:102C1000430F09E041EA030C50EA4C0C52EA0C0C59
:102C200003D28B4208BF8242704714BF9942904240
:102C30007047000070B504460D466068C0F30A5046
:102C400040F2FF72904207D16068000304BF206821
:102C5000002817D0022070BD20B92046FFF799FF49
:102C6000012867DA012D0FDB40F2FF71091A8D424E
:102C70000AD36068002847BF00202F4900202F4951
:102C8000C4E90001012070BD4142A942616806DA31
:102C90006FF31E51401941EA0050606041E001F0BD
:102CA00000410122636862F31F536360401E4519AF
:102CB00005F13500352803D361600020206070BD28
:102CC000002215F11F0F04DA20352268236000204E
:102CD0006060684213D0521E9241D243C0F120037B
:102CE00025689D4055EAD2722568C540666806FA97
:102CF00003F32B432360636823FA00F0606060688D
:102D000008436060B2F1004F03D80DD12078C007AE
:102D10000AD52068401C2060206828B96068401CE3
:102D200060604FF0FF3070BD6068884204BF20686B
:102D30000028F6D1002070BD0000F0FF0000F07FF9
:102D4000F446400D40EAC120490006D200F014F8D4
:102D5000004248BF6FF00040604700F00DF84FF0B0
:102D6000004188428CBF084640426047400D40EA1F
:102D7000C120490080F00D8040F00040490DA1F5D0
:102D80008061491C05D4D1F11F0154BFC840C01750
:102D900070474FF000007047010040F10980F44691
:102DA000404200F005F851F000416047010000BFCB
:102DB00009D0B0FA80F18840C91CC1F584610905C9
:102DC00001EBD0214005704770B44FF0004591EA07
:102DD000030F44BF6B4000F03BBB00BF841A71EB94
:102DE000030604D26E40001BB141121973414FF427
:102DF000001C1CEB410F34BF7CEB430684E00C0D40
:102E0000A4EB1356362E7DDC012E43DC45EAC323AA
:102E100043EA525312BFD20292025B08240545EAEC
:102E2000C12141EA5051D2EBC020994125D407D1AC
:102E3000B0FA80F610FA06F164D00020203608E0DF
:102E4000B1FA81F6B140C6F1200220FA02F2114334
:102E5000B0404FEAF474B4EB465434F001064FEA44
:102E600074040AD8D6F50016760D04F00044F0403C
:102E700061FA06F25040F1404840C00A40EA415031
:102E800021F0004128BF5FEA500550F1000044EBFB
:102E9000D12137E045EAC323DB0A45EAC121C90A4B
:102EA000B6F120050EDD42EA0242120CC5F1200601
:102EB00003FA06F6EB4042EA06056D42984161F1DD
:102EC00000010DE062FA06F5F240554063FA06FC97
:102ED00082EA0C02F3405A406D42904161EB0301DB
:102EE00011F4801F05D1641E620502D06D004041BF
:102EF000494121F48011430875F1004350F100006D
:102F000041EB045170BC70471CEB410F15D223F00C
:102F1000004352EA43060BD04FEA4C0CBCEB410F86
:102F200004D80C0D661E342EB7DDEBE7801A9941EC
:102F300050EA410608BF0021E4E708BF1CEB430F3D
:102F400028BF6FF00001DDE7B0B581EA030C0CF09B
:102F5000004C40F2FF7515EA11541DBF15EA1357D6
:102F6000AC42AF4239E0E41923EA455343F48013FD
:102F7000C90241F0004141EA505EC7021100A7FBBF
:102F8000020200284FF00000EEFB01204FF000018C
:102F9000E3FB072118BF42F001024018002149411C
:102FA000E3FB0E01A4F580640F0302D252004041FE
:102FB000494154F101046CDD470872F1004250F1BF
:102FC000000051EB0451A1F580115CBF41EA0C01F6
:102FD000B0BD4CEA05510020B0BD05EA1357AC4224
:102FE00014BFAF4241E050EA410E1CBF52EA430E0B
:102FF00002E061460020B0BD24423C441BD15FEAA0
:10300000070EF6D0090302BF01460020AEF1140EF0
:10301000B1FA81F7AEEB070401FA07FE0C37C7F1EE
:10302000200100FA07F7C8404EEA000E23EA455394
:1030300043F48013A2E733F00043B3FA83F704BFED
:10304000B2FA82FE77440B3FE41BB7F1200E2FBF8C
:1030500002FA0EF3BB40C7F1200E22FA0EFE38BF73
:1030600043EA0E03BA40641C82E750EA410E14BFE3
:1030700052EA430E6FF000014FF4001717EB430FB5
:103080008ABF194617EB410FB5E74CEA05510020FE
:10309000B0BDD4F10104B4F120070FDAC4F1200768
:1030A000520828BF42F0010210FA07F501FA07F7AB
:1030B000E1BF2A43E0403843E1400FE0352C98DC83
:1030C000C7F1200452EA400220FA07F218BF42F08A
:1030D000010231FA07F0A1400A43002172F10042D7
:1030E00050F1000051EB0C01B0BD0000F0B540F212
:1030F000FF7581EA030C0CF0004C15EA11541DBF5A
:1031000015EA1357AC42AF42E5E0BC41C1F31301ED
:10311000C3F31303801A994143F4801304D2641E4D
:103120004000494180185941C90241EA5051B1FB60
:10313000F3F603FB1611A2FB0675D7EBC020A941DD
:1031400002D2761E80185941C90241EA5051B1FBA2
:10315000F3FE03FB1E11A2FB0E75D7EBC020A941A5
:1031600003D2AEF1010E80185941890241EA905113
:10317000760546EA8E2EB1FBF3F603FB1611A2FB91
:103180000675D7EB8020A94102D2761E80185941DE
:10319000C90241EA50514EEA060EB1FBF3F603FBB9
:1031A0001611A2FB0675D7EBC020A94102D2761EEC
:1031B00080185941C90241EA5051B1FBF3F703FBB2
:1031C0001711A2FB0735D3EBC020A94167F1000717
:1031D0000CBF004247F0010766F3D5274FEA1E31C6
:1031E000B80814F5806412DDBD0775F1004250EB9C
:1031F0000E5051EB045111F5801F5CBF41EA0C01E8
:10320000F0BD4CF07F6141F0E0410020F0BDBD0712
:103210006D0840EA0E5041F48011D4F10104B4F17C
:1032200020060ADAC4F120060200E04001FA06F3A3
:10323000E1401843B24015430EE0342C13DCC6F1D4
:10324000200445EA40056D0820FA06F2154321FAEC
:1032500006F0A1400D43002175F1004250F100003D
:1032600051EB0C01F0BD00205FEA0C01F0BDCFB9BD
:1032700092185B41B3FA83F704BFB2FA82F6BF1922
:103280000B3FB7F120062FBF02FA06F3BB40C7F190
:10329000200622FA06F638BF3343BA401CB1E419BF
:1032A000641E33E77F4231F00041B1FA81F404BF7C
:1032B000B0FA80F6A4190B3CB4F120062FBF00FA37
:1032C00006F1A140C4F1200620FA06F638BF3143CA
:1032D000A0403C1B1AE7AC421ABF05EA1357AF42A5
:1032E00012E050EA41061CBF52EA4306BFE750EA2B
:1032F0004107304661461CBF41EA0551F0BD52EA24
:10330000430C08BFC143F0BD00204FF4001616EB7C
:10331000410F98BF16EB430F08BF16EB410F24BFB8
:10332000C14305E016EB430F0CBF61464CEA055163
:10333000F0BD000080B5134800F0F4F80FF248012A
:10334000016041608160C1600161416181610FF292
:103350003C0242628162C162016341630FF230024A
:1033600082630FF23402C2630164416401BD10B58F
:10337000044800F0D7F80446206808B9FFF7DAFFE0
:10338000204610BD20030020000000002E00000099
:1033900066616C7365000000747275650000000062
:1033A00091FBF2F303FB1211C0E9003170470000FA
:1033B00080B5DFF80C0000F0B5F8806902BD0000B0
:1033C0005C0D002030B430B90FF24800D0E9004560
:1033D000C2E900451BE00170012030BC704730B4E9
:1033E00031B90FF23800D0E90045C3E900450EE0DD
:1033F0001AB96FF0010030BC704708B10A7802803A
:103400000978481E8041C043C00F30BC704700207F
:1034100030BC704700000000000000000000000009
:10342000000000000649086808B100207047054800
:1034300008600549C908C900091A0160704700BF42
:10344000000E0020080E0020081600207047000023
:10345000841A71EB030603D2001BB14112197341A8
:103460004FF4001C1CEB410F34BF7CEB430443E0E2
:103470000C0DA4EB1356352E50DC45EAC323DB0AB2
:1034800045EAC121C912B6F120050DDD63FA05F642
:10349000EB4086EA0305124218BF45F00105C0184B
:1034A00051F100010CD213E062FA06F5F2405540EA
:1034B000F3415A40B340F3405A408018594107D372
:1034C00049085FEA30005FEA350528BF45F001058D
:1034D00001F58011420875F1004250F1000041EB06
:1034E000045170BC4FF4001C1CEB410F38BF7047F7
:1034F0000020090D090570471CEB410F10D252EA5C
:1035000043060BD0BCEB410F05D80C0DAB43661E38
:10351000342EB5DD02E0AB438018594170BC7047D2
:1035200070BC70477047000010B5074979441831E6
:10353000064C7C44163404E0081D0A68511888477C
:103540000146A142F8D110BD08000000280000008B
:10355000ABE1FFFF940A00007003002000000000B0
:103560000BDEFFFF70030000900100000000002050
:103570000000000000F009F8002801D0FFF7D4FF98
:103580000020FDF761FC00F002F80120704700F018
:1035900001B800000746384600F002F8FBE70000DB
:1035A000C046C046024A11001820ABBEFBE700BF70
:1035B0002600020020D2E5EA207C20CCE0EAF17C63
:1035C00020CCE8ED2000000020CAE0EBE8E1F0EEBE
:1035D000E2EAE02E2E2E2000D1C1CEC920EAE0EB97
:1035E000E8E1F0EEE2EAE800253469207C25346960
:1035F000207C2534690000000148804701480047CD
:103600004901000815360008C2E8EBEAE02025343D
:1036100069560000C046C046C046C046FFF7AAFF34
:10362000253469C200000000FCF7F8BEFCF7F7BEC5
:10363000FCF7F6BEFCF7F5BEFCF7F4BEFCF7F3BEF4
:10364000FCF7F2BEFCF7F1BEFCF77ABFFFF7FEBF56
:10365000FFF7FEBFFFF7FEBFFFF7FEBFFFF7FEBF9E
:10366000FFF7FEBFFFF7FEBFFFF7FEBFFFF7FEBF8E
:10367000FFF7FEBFFFF7FEBFFDF76DBBFFF7FEBF15
:10368000FFF7FEBFFFF7FEBFFFF7FEBFFFF7FEBF6E
:10369000FFF7FEBFFFF7FEBFFFF7FEBFFFF7FEBF5E
:1036A000FFF7FEBFFFF7FEBFFFF7FEBFFFF7FEBF4E
:1036B000FFF7FEBFFFF7FEBFFFF7FEBFFFF7FEBF3E
:1036C000FFF7FEBFFFF7FEBFFFF7FEBFFFF7FEBF2E
:1036D000FFF7FEBFFFF7FEBFFFF7FEBFFFF7FEBF1E
:1036E000FFF7FEBFFFF7FEBFFFF7FEBFFFF7FEBF0E
:1036F000FFF7FEBFFFF7FEBF000000000000005F05
:1037000000000007000700147F147F14242A7F2A7A
:103710001223130864623649552250000503000045
:10372000001C2241000041221C0014083E0814081D
:10373000083E08080050300000080808080800602B
:1037400060000020100804023E5149453E00427FBF
:10375000400042615149462141454B311814127FC6
:103760001027454545393C4A49493001710905034F
:103770003649494936064949291E003636000000B7
:103780005636000008142241001414141414004189
:103790002214080201510906324979413E7E111175
:1037A000117E7F494949363E414141227F414122B4
:1037B0001C7F494949417F090909013E4149497A2C
:1037C0007F0808087F00417F41002040413F017F82
:1037D000081422417F404040407F020C027F7F045A
:1037E00008107F3E4141413E7F090909063E415193
:1037F000215E7F09192946464949493101017F0166
:10380000013F4040403F1F2040201F3F4038403F85
:1038100063140814630708700807615149454300A1
:103820007F41410002040810200041417F00040252
:103830000102044040404040000102040020545472
:1038400054787F48444438384444442038444448F9
:103850007F3854545418087E0901020C5252523ECB
:103860007F0804047800447D40002040443D007FF0
:103870001028440000417F40007C041804787C0834
:1038800004047838444444387C141414080814148C
:10389000187C7C080404080854545420043F444015
:1038A000203C4040207C1C2040201C3C4030403CC0
:1038B00044281028440C5050503C4464544C44005C
:1038C0000836410000007F00000041360800100863
:1038D00008100878464146787E1111117E7F4949CB
:1038E00049317F494949367F01010103603E212169
:1038F0007F7F4949494177087F0877224149493606
:103900007F1008047F7F1009047F7F081422414044
:103910003E01017F7F020C027F7F0808087F3E4145
:1039200041413E7F0101017F7F090909063E414176
:10393000412201017F0101274848483F1E217F2184
:103940001E63140814633F20203F60070808087FA7
:103950007F407F407F3F203F207F017F4848307F6E
:103960004830007F007F484830224149493E7F0867
:103970003E413E462919097F20545454783C4A4A16
:103980004A307C545428007C040404046038242405
:103990007C38545454186C107C106C0044545428D7
:1039A0007C2010087C7C2112097C7C10284400407B
:1039B0003804047C7C0810087C7C1010107C38448F
:1039C0004444387C0404047C7C14141408384444B3
:1039D000440004047C04040C5050503C08147C1433
:1039E0000844281028443C20203C600C1010107C17
:1039F0007C407C407C3C203C207C047C5050207CE3
:103A00005020007C007C50502028445454387C10B6
:103A1000384438485434147C000000000000000092
:103A20000000000000000000000000000000000096
:103A300000000000FFFFFFFFFFFFFFFF000000008E
:103A40000000000000000000000000000000000076
:103A50000000000000000000000000000000000066
:083A6000FFFFFFFFFFFF000064
:0400000508003615A4
:00000001FF
